:10000000000008308A00F12EFF00030E8312031354
:10001000A1000A08A0008A010408A2007708A30032
:100020007808A4007908A5007A08A6007B08A70034
:10003000831383128B1E1E280B193128220884007B
:100040002308F7002408F8002508F9002608FA001C
:100050002708FB0020088A00210E8300FF0E7F0E78
:1000600009008A110A1273290A108A100A118207DC
:100070006D346F3474346F3472345F3463346F347E
:1000800075346E347434733420343D342034253464
:100090006C3464340D340A3400340A108A100A11A6
:1000A00082070A3400340A108A100A118207453484
:1000B00052345234203425343234583425343234D6
:1000C00058340D3400340A108A100A118207523451
:1000D000443459340D3400340A108A100A1182074E
:1000E000533454344F3450345F3450344F345334D9
:1000F000203425346C3464340D3400340A108A10F2
:100100000A1182075334543441345434553453342F
:1001100020343034783425343034323458340D348B
:1001200000340A108A100A11820750344F345334B5
:100130004934543449344F344E34203425346C34EB
:1001400064340D3400340A108A100A1182072034F6
:1001500000340A108A100A1182074F345034453493
:100160004E3400340A108A100A11820743344C348A
:100170004F345334453400340A108A100A11820770
:100180004D344F345634453400340A108A100A1165
:1001900082075334453454345F34533454344F3429
:1001A000503400340A108A100A118207473445344B
:1001B00054345F34533454344F34503400340A10C0
:1001C0008A100A1182074A344F3447345F344F345F
:1001D00000340A108A100A1182074A344F34473417
:1001E0005F34433400340A108A100A1182074734FE
:1001F000453454345F3450344F34533400340A148B
:100200008A100A1182074734453454345F3453341A
:1002100054344134543400340A148A100A118207C9
:100220004534433448344F3400340A148A100A11D8
:10023000820743344C3452345F3450344F34533497
:1002400000340A148A100A118207533448344F3498
:1002500057345F3443344E345434533400348316AB
:100260003E0840068039C200BE1B382983123E2951
:10027000BD09BE09BD0A0319BE0A83128316C01B3D
:10028000432983124929BF09C009BF0A0319C00ABB
:1002900083121030F700FA018316C101831283160E
:1002A000BE0CBD0C0318562983125D293F08FA07BE
:1002B0000318C10A4008C10783128316C10CFA0C47
:1002C000F90CF80CF70B6529672983124F29C21B1B
:1002D0006B2983127129F809F909F80A0319F90A37
:1002E000831200000034891083168910FF308800C3
:1002F0008312310808028316BC0083128914831606
:1003000089103C088039003A031D882983129C29F2
:10031000831283163C08FF3A013E8312B10200307B
:10032000031C0130B2020030031C0130B302003064
:10033000031C0130B402AC2983163C088312B107B8
:10034000003003180130B207003003180130B30742
:10035000003003180130B407FA0183163C08F70097
:10036000F71BFA038312B5007A08B6003608831625
:10037000BE00831235088316BD00C0013D30BF00AA
:1003800083122F217908B6007808B500B70A03193F
:10039000B80A0B118A110A121E288B128101B801AA
:1003A000B7018B1600348B120911831609118312C1
:1003B0000915831609118312B401B301B201B10109
:1003C0008B16003403178D018F0183168C130C14C8
:1003D00083120C080313C300013003178D008F0133
:1003E00083168C130C1483120C080313C400023000
:1003F00003178D008F0183168C130C1483120C08C5
:100400000313C500033003178D008F0183168C136F
:100410000C1483120C080313C6004308BE004408E2
:10042000BD004508BC004608BB00043003178D0022
:100430008F0183168C130C1483120C080313C30052
:10044000053003178D008F0183168C130C14831253
:100450000C080313C400063003178D008F018316A8
:100460008C130C1483120C080313C50007300317F8
:100470008D008F0183168C130C1483120C08031348
:10048000C6004308C2004408C1004508C000460831
:10049000BF003F083B02031D5C2A40083C02031DCD
:1004A0005C2A41083D02031D5C2A42083E02031DEE
:1004B0005C2A0130AF005D2AAF013B08F7003C0821
:1004C000F8003D08F9003E08FA008A150A12462F86
:1004D0008C1E682A1808A8001A08F800A81C722A9E
:1004E0001812181600000034E801831686148312CF
:1004F000861C6814831606168312061EE8148316DB
:1005000086168312861E6815B008031DE815680854
:10051000F8000034EA1B9D2A0F30F700690EF7053A
:100520000A3077020318972A3030F707992A6A08A9
:10053000F70777080C1E9A2A99000F30E9050A3050
:1005400069020318A52A3030A72AEA136A08E907C6
:1005500069080C1EA92A9900003474227808E70063
:10056000E608031DB82A67080139003A0319D22AA0
:10057000E80168085320E80A0C1EBC2A99000430E0
:100580006802031DB92A6708E9003730EA008A22A9
:100590006608E9003730EA008A220D300C1ECE2AA8
:1005A0009900DD2AE80168086320E80A0C1ED62AB3
:1005B000990004306802031DD32AB9080319E42AFC
:1005C0000A300C1EE12A99000034DC080319EA2ADB
:1005D0005C08EB2A2908DE005E08E0005D08E10007
:1005E0006008E2006208840080080319112B61088A
:1005F000E300630884008008031D032B6008620287
:10060000F800142B0D2B620884000008E400630836
:1006100084000008640203190F2BE30AF92AE20A96
:10062000F22A60086202F8007808DE075E0884009B
:100630008008031D222B2908840020308000003010
:10064000F800562B5E08E0005D08E1006008E2005B
:100650006208840080080319452B6108E3006308E1
:10066000840080080319432B620884000008E4001A
:100670006308840000086402031D412B6208F8002F
:10068000472BE30A2F2BE20A282B0030F8007808CA
:10069000DF005F08840080080319522B5F08840084
:1006A0008001DF0A5F08A9005E08F80000345C08DA
:1006B00084000008DE005D08840000085E02031963
:1006C0009F2B5C0884000008DF005F08403C031893
:1006D0006D2B5F085A3C0318752B5F08603C0318AC
:1006E000AB2B5F087A3C031CAB2B5D088400000831
:1006F000E0006008403C0318812B60085A3C031856
:10070000892B6008603C0318AB2B60087A3C031C03
:10071000AB2B5C0884000008E1005D0884002030F9
:100720000007610203199F2B5D0884000008E300A5
:100730005C088400203000076302031DAB2B5C08BB
:1007400084008008031DA72B0030F800B92B5C083B
:10075000DC0ADD0A572B5C0884000008DE005D0817
:10076000840000085E020318B72BFF30B82B01305D
:10077000F8000034F701F801F901FA018316AE011F
:10078000AF01B001B1012D082C042B042A04031D74
:10079000CB2B83120D2C831220308316B2008312D0
:1007A00003108316A60DA70DA80DA90DAE0DAF0D54
:1007B000B00DB10D2D0831020319E02B8312EF2B80
:1007C0002C0830020319E62B8312EF2B2B082F0283
:1007D0000319EC2B8312EF2B2A082E028312031C21
:1007E000022C83162A08AE022B08031C2B0FAF0223
:1007F0002C08031C2C0FB0022D08031C2D0FB10276
:1008000003148312F70DF80DF90DFA0D8316B20BD0
:100810000A2C0C2C8312D02B83120000AE308400E3
:10082000003404088316A000F51B182C8312282C12
:100830002D3083120C1E1A2C9900F209F309F409C9
:10084000F509F20A0319F30A0319F40A0319F50A60
:100850003B308316A5009A30A400CA30A300A20141
:100860000A30A100831275088316A9007408A80035
:100870007308A7007208A6002508AD002408AC0084
:100880002308AB002208AA008312BA230008F20052
:10089000840A0008F300840A0008F400840A0008AF
:1008A000F500FD308407F708031D742C831621081A
:1008B000013A031D5D2C8312742C2008031D622C49
:1008C0008312772C0F392102031D682C83126D2CA3
:1008D000031C6C2C83127D2C8312F0308316201B9A
:1008E0000030F7008312772C8316A001831230307A
:1008F000F70777080C1E7A2C990083162508A900A3
:100900002408A8002308A7002208A600AD01AC0116
:10091000AB010A30AA008312BA237A088316A50015
:100920007908A4007808A3007708A200A10B992CED
:100930009B2C8312332C83120034EF01660831079D
:10094000EA003208EB0067080318670FEB0733086B
:10095000EC0068080318680FEC073408ED0069081C
:100960000318690FED07B41FB82CED1BBA2CD02C5F
:10097000ED1BE72C34086D02031CE72C031DD02C63
:1009800033086C02031CE72C031DD02C32086B02C9
:10099000031CE72C031DD02C6A0831020318E72C36
:1009A0000130EE0007113A113A08831687008312CE
:1009B0008714BA103A088316870083120516831627
:1009C000051283128512831685128312FC2CEE0108
:1009D00007153A113A088316870083128710BA1058
:1009E0003A088316870083120512831605128312B4
:1009F0008516831685128312CD213608FA00350834
:100A0000B61F0B2D3508003CF700FA013608031C11
:100A1000360FFA027708F1007A08F200F21F112D62
:100A2000182DF208031D202D7108C73C031C202D32
:100A3000B808031D202D3708063C031C202DFD2C73
:100A40006E0B482DED1F272DB41B292D3E2DB41BF9
:100A50003F2D6D083402031C3F2D031D3E2D6C08F5
:100A60003302031C3F2D031D3E2D6B083202031C75
:100A70003F2D031D3E2D31086A02031CB32D831642
:100A800006168312061A472D0730EF00B32D6D2D81
:100A9000B41F4D2DED1B4F2D642DED1B652D34081E
:100AA0006D02031C652D031D642D33086C02031CAD
:100AB000652D031D642D32086B02031C652D031D7B
:100AC000642D6A083102031CB32D83168616831227
:100AD000861A6D2D0830EF00B32D8C1E732D682201
:100AE0000630EF00B32D3608FA003508B61F812D09
:100AF0003508003CF700FA013608031C360FFA02ED
:100B00007708F1007A08F200F21F872D8E2DF20887
:100B1000031D912D7108C73C031C912D0930EF0076
:100B2000B32DAA080319B22DF10171083420F10A7E
:100B30000C1E982D99000F307102031D952D413028
:100B400084003408F5003308F4003208F30031085B
:100B5000F20011240D300C1EAB2D99000A300C1E32
:100B6000AF2D9900202D07113A113A0883168700FE
:100B700083128710BA103A08831687008312051271
:100B800083160512831285128316851283126F084D
:100B9000F8000034DC01B008031DD22D0A30E60055
:100BA000AD22FC2DAF08031DD92D0B30E600AD2280
:100BB000FC2D31082B02DD002C08DE003208031C5E
:100BC000320FDE022D08DF003308031C330FDF0273
:100BD0002E08E0003408031C340FE0026008E9002E
:100BE0005F08E8005E08E7005D08E6009D247808DD
:100BF000DC005C08E600AD228A150A12832D5D3008
:100C0000840000080319132E0130F800F701F70BD8
:100C1000072EF80B062E4A30F700F70B0D2E0000BA
:100C20000000800B042E8A110A129F2EDC01742210
:100C300078080439003A0319232E0130B000D3217B
:100C4000E601AD22AC2E07153A113A08831687004B
:100C500083128710BA103A08831687008312051290
:100C60008316051283128516831685128312CD21F1
:100C70003608FA003508B61F462E3508003CF70046
:100C8000FA013608031C360FFA027708DD007A08ED
:100C9000DE00DE1F4C2E532EDE08031D5B2E5D088A
:100CA000C73C031C5B2EB808031D5B2E3708063CAF
:100CB000031C5B2E382E8C1E612E68220630DC0051
:100CC000882E831686168312861A692E0830DC0059
:100CD000882E3608FA003508B61F772E3508003CF6
:100CE000F700FA013608031C360FFA027708DD0018
:100CF0007A08DE00DE1F7D2E842EDE08031D872E7F
:100D00005D08C73C031C872E0930DC00882E5B2E53
:100D100007113A113A088316870083128710BA1018
:100D20003A08831687008312051283160512831270
:100D30008512831685128312C830DD00FF2D5C08F2
:100D4000083C031DA92E0130B000D321E601AD22DD
:100D5000AC2E5C08E600AD228A150A12A22D0130E5
:100D6000E700E80166086807840080080319CF2EB1
:100D70006808E80A660784000008EA006A082B3C55
:100D80000319CE2E6A082D3C0319CE2E6A082F3C7B
:100D90000318CD2E6A08393C031CE701B22E670800
:100DA000F80000346608E70067088400800803192B
:100DB000DB2EE70AD42E66086702F8000034EB0148
:100DC000E9010A30EA00E801E7016B08EB0A66076F
:100DD00084000008EC006C082F3C0318F32E6C080C
:100DE000393C0318FB2E6C082B3C0319FB2E6C08B6
:100DF0002D3C031DE52E6C082D3C031D082F0130F2
:100E0000E9006B08EB0A660784000008EC00122F6B
:100E10006C082B3C031D122F6B08EB0A660784003D
:100E20000008EC006C082F3C0318C42F6C08393CF8
:100E3000031CC42F6C08303C031D352F66086B075C
:100E400084000008783C03192C2F66086B07840087
:100E50000008583C031D352F1030EA00EB0A6B08E0
:100E6000EB0A660784000008EC006A080A3C031DD0
:100E7000692F6C082F3C0318682F6C08393C031C41
:100E8000682F8316BE010A30BD00831268088316DE
:100E9000C000831267088316BF0083120B080B057E
:100EA0008B13A0002F2120088B047908EE0078080E
:100EB000ED0030306C026D07E7006E08E8000318A3
:100EC000E80A6B08EB0A660784000008EC00392F7B
:100ED000C42F6A08103C031DC42F6C08603C031823
:100EE000782F6C087A3C031C782F6C08DF39792F37
:100EF0006C08EC002F3C0318812F6C08393C031858
:100F0000892F6C08403C0318C42F6C08463C031C16
:100F1000C42F6C082F3C0318A72F6C08393C031C06
:100F2000A72F0310670DED00680DEE00ED0DEE0D1F
:100F3000ED0DEE0DED0DEE0DF030ED0530306C02E7
:100F40006D07E7006E08E8000318E80ABD2F0310DC
:100F5000670DED00680DEE00ED0DEE0DED0DEE0DE3
:100F6000ED0DEE0DF030ED0541306C020A3E6D07DF
:100F7000E7006E08E8000318E80A6B08EB0A66074A
:100F800084000008EC006D2F6A080A3C031DCF2F77
:100F9000690BCF2FE709E809E70A0319E80A670890
:100FA000F8006808F90000342030EC00E801E9019D
:100FB000EA01EB016308FA006208F9006108F80031
:100FC0006008F7000310771CF32F6408E807650832
:100FD0000318650FE90766080318660FEA07670834
:100FE0000318670FEB07EB0CEA0CE90CE80CFA0CA2
:100FF000F90CF80CF70CEC0BE22F8A150A12792B7E
:1010000069086D068039F600E91F1128E609E7092D
:10101000E809E909E60A0319E70A0319E80A0319C6
:10102000E90AED1F1E28EA09EB09EC09ED09EA0AB5
:101030000319EB0A0319EC0A0319ED0A2030F50035
:10104000F101F201F301F4016908FA006808F900FE
:101050006708F8006608F7000310771C3D286A0847
:10106000F1076B0803186B0FF2076C0803186C0F7D
:10107000F3076D0803186D0FF407F40CF30CF20C72
:10108000F10CFA0CF90CF80CF70CF50B2C28F61FE8
:101090005428F709F809F909FA09F70A0319F80AAF
:1010A0000319F90A0319FA0A00346D087406803925
:1010B0008316A5008312ED1F6828EA09EB09EC09E5
:1010C000ED09EA0A0319EB0A0319EC0A0319ED0A00
:1010D000F41F7528F109F209F309F409F10A03195B
:1010E000F20A0319F30A0319F40AF701F801F901E6
:1010F000FA018316A001A101A201A30174087304DF
:1011000072047104031D86288312C82883122030BC
:101110008316A40083120310EA0DEB0DEC0DED0D08
:101120008316A00DA10DA20DA30D740823020319AF
:101130009B288312AA28730822020319A12883126C
:10114000AA28720821020319A7288312AA28710865
:1011500020028312031CBD2871088316A0027208A6
:10116000031C720FA1027308031C730FA202740800
:10117000031C740FA30203148312F70DF80DF90D6D
:10118000FA0D8316A40BC528C72883128B28831257
:1011900000008316A51BCE288312DA28F709F80968
:1011A000F909FA09F70A0319F80A0319F90A0319E0
:1011B000FA0A8312A030840000345C08E6008A1129
:1011C000AF268A15F808031DEB280230E6008A11C5
:1011D000AD228A1597295C08E6008A11D2268A1565
:1011E0007808053C0318FA280330E6008A11AD227E
:1011F0008A159729DC08031D03290430E6008A11AB
:10120000AD228A1597295C08E6008A11DF268A1527
:101210007808F7007908F800F901FA01F81F122997
:10122000F903FA037A08E1007908E0007808DF00A2
:101230007708DE005E08F7005F08F8006008F90034
:101240006108FA00E11F36295E08003CF700F8014A
:101250005F08031C5F0FF802F9016008031C600FB0
:10126000F902FA016108031C610FFA027A08E90029
:101270007908E8007808E7007708E600E91B5729B5
:10128000E908031D5129E808031D51296708023C9C
:1012900003185729FF3A031D51296608E83C031833
:1012A00057290530E6008A11AD228A159729E901F0
:1012B000E8010F30E7006030E6006108ED006008EB
:1012C000EC005F08EB005E08EA0000207A08E90005
:1012D0007908E8007808E7007708E6006908ED007B
:1012E0006808EC006708EB006608EA00F401F30107
:1012F0000330F200E830F10055207A08E500790863
:10130000E4007808E3007708E2006508E900640873
:10131000E8006308E7006208E6008A119D248A1548
:101320007808DD005D08E6008A11AD228A158A156D
:101330000A12CA2DB008031DA3290A30E6008A113B
:10134000AD228A15662B5C08E6008A11AF268A1545
:10135000F808031DB1290230E6008A11AD228A1572
:10136000662B5C08E6008A11D2268A157808053CAF
:101370000318C0290330E6008A11AD228A15662BB6
:10138000DC08031DCC293408E4003308E3003208EC
:10139000E2003108E100112A5C08E6008A11DF262C
:1013A0008A157808F7007908F800F901FA01F81FA2
:1013B000DB29F903FA037A08E0007908DF007808EE
:1013C000DE007708DD00E901E8010F30E70060305A
:1013D000E6006008ED005F08EC005E08EB005D08C9
:1013E000EA0000207A08E8007908E7007808E600BB
:1013F0007708E5006808ED006708EC006608EB0078
:101400006508EA00F401F3010330F200E830F1006E
:1014100055207A08E4007908E3007808E2007708AC
:10142000E100E41F142A152A192AE401E301E2016C
:10143000E1016408E8006308E7006208E60061086B
:10144000E5006808E90003178D018F01031369089F
:1014500003178C0083168C130C15831203130B08CF
:10146000F7008B135530831603178D00AA308D00BB
:101470008C1483120313831603178C1C422A8312C5
:1014800003133B2A0C117708831203138B0467089C
:10149000E900013003178D008F010313690803175A
:1014A0008C0083168C130C15831203130B08F700A2
:1014B0008B135530831603178D00AA308D008C14C2
:1014C00083120313831603178C1C692A83120313D8
:1014D000622A0C117708831203138B046608E90053
:1014E000023003178D008F010313690803178C0066
:1014F00083168C130C15831203130B08F7008B1340
:101500005530831603178D00AA308D008C1483127A
:101510000313831603178C1C902A83120313892A42
:101520000C117708831203138B046508E90003305C
:1015300003178D008F010313690803178C008316AE
:101540008C130C15831203130B08F7008B13553003
:10155000831603178D00AA308D008C148312031399
:10156000831603178C1CB72A83120313B02A0C119D
:101570007708831203138B046808E900043003170B
:101580008D008F010313690803178C0083168C13D9
:101590000C15831203130B08F7008B1355308316B9
:1015A00003178D00AA308D008C1483120313831649
:1015B00003178C1CDE2A83120313D72A0C11770819
:1015C000831203138B046708E900053003178D00AD
:1015D0008F010313690803178C0083168C130C15F5
:1015E000831203130B08F7008B1355308316031770
:1015F0008D00AA308D008C148312031383160317F9
:101600008C1C052B83120313FE2A0C1177088312FE
:1016100003138B046608E900063003178D008F0161
:101620000313690803178C0083168C130C1583129F
:1016300003130B08F7008B135530831603178D0027
:10164000AA308D008C1483120313831603178C1C8D
:101650002C2B83120313252B0C11770883120313F1
:101660008B046508E900073003178D008F01031311
:10167000690803178C0083168C130C15831203134F
:101680000B08F7008B135530831603178D00AA3013
:101690008D008C1483120313831603178C1C532B99
:1016A000831203134C2B0C117708831203138B0442
:1016B0006408AE006308AD006208AC006108AB00CE
:1016C0000130AF00E6018A11AD228A158A150A128F
:1016D000F12D2E08E3002D08E2002C08E1002B0874
:1016E000E000E701E6010330E500E830E4008A119C
:1016F000D42F8A157A08E3007908E2007808E1001F
:101700007708E00063088316A90083126208831635
:10171000A800831261088316A7008312600883164D
:10172000A600AD01AC010F30AB006030AA008312FF
:101730008A11BA238A157A08DF007908DE00780852
:10174000DD007708DC00E00160088A116C208A1552
:10175000E00A0C1EA92B990009306002031DA42B7E
:10176000413084005F08F5005E08F4005D08F30076
:101770005C08F2008A1111248A150D300C1EBE2B54
:101780009900B9080319C82B0A300C1EC52B990003
:10179000E6018A11AD228A158A150A120E2E5C0BFB
:1017A000DE2BE9010130E8008630E700A030E600DA
:1017B0008A119D248A157808DD00EB2BFF30E900A3
:1017C000FE30E8007930E7006030E6008A119D24A1
:1017D0008A157808DD005D08E6008A11AD228A15B9
:1017E00000340408E600E01FFF2B2D300C1EF62B02
:1017F00099008403DF09E009DF0A0319E00A600E9B
:10180000F038E200E207E23EE300323EE500600825
:101810000F39E307E307E507E93EE400E407E407DF
:101820005F0E0F39E407E507E40DE50DE509E50D69
:101830005F080F39E507E20D0730E1000A30E507E0
:10184000E403031C1F2CE407E303031C232CE3071E
:10185000E203031C272CE207E103031C2B2C61305D
:1018600084000730660584076530040203194C2C98
:101870000008F700031D422C661A4A2CE619442C76
:101880002030452C0830E6003030F70777080C1E72
:10189000472C9900840A342C0008F7003030F707F1
:1018A00077080C1E512C99008A150A129E2CB0083C
:1018B000031D602C0A30E6008A11AD228A15AD2C7A
:1018C0003408E9003308E8003208E7003108E60090
:1018D000ED01EC010330EB00E830EA0000207A086B
:1018E000E1007908E0007808DF007708DE00610891
:1018F000ED006008EC005F08EB005E08EA00F40110
:10190000F3010F30F2006030F10055207808DD005F
:101910007708DC00DE015E088A1191208A15DE0A54
:101920000C1E902C990009305E02031D8B2C103088
:1019300084005D08E0005C08DF00F12B0D300C1E18
:101940009F2C9900B9080319A92C0A300C1EA62C4B
:101950009900E6018A11AD228A158A150A12682EAD
:101960008A1174228A157808DC00DD015D088A116D
:101970007E208A15DD0A0C1EBB2C990009305D0201
:10198000031DB62C5C08E9003730EA008A118A2270
:101990008A150D300C1ECA2C9900B9080319D42CD5
:1019A0000A300C1ED12C9900E6018A11AD228A154D
:1019B0008A150A12852EB9080319E02C0030E12C93
:1019C0000130B900E6018A11AD228A158A150A1282
:1019D000A22EDD01DC015A3084005C0884075D081A
:1019E0008A11A3208A15800000380319FA2CDD0A19
:1019F000DC0AEB2C3C30DC000F30DD00DD03DE01C7
:101A00008A1168228A157808DF00083C031D1C2D06
:101A1000DE0803191B2DDE03B90803191B2D5F080F
:101A20000C1E102D990020300C1E142D99005F08FB
:101A30000C1E182D9900352D5F081F3C0318352DFD
:101A40005F087E3C031C352D5D085E020318352DB2
:101A50005E08DE0A5C0784005F088000B90803198D
:101A6000352D5F080C1E322D99005F080D3C031DBB
:101A7000002D5C085E0784008001B9080319552D0C
:101A8000E00160088A114D208A15003803194D2D98
:101A9000E00A0C1E492D9900412D0D300C1E4E2DD3
:101AA00099000A300C1E522D9900BC08031D5D2DB3
:101AB000E6018A11AD228A15EE2E3C30DC005A3048
:101AC000DD008A11E5228A157808BB00DD01DC0102
:101AD0004B3084005C0884075D088A11A9208A15B0
:101AE000800000380319772DDD0ADC0A682D3B08D9
:101AF000DC004B30DD008A1157238A15F808031DDE
:101B0000852D8A11CA2D8A15EE2EDD01DC014B30A0
:101B100084005C0884075D088A11B2208A15800061
:101B200000380319962DDD0ADC0A872D3B08DC00FE
:101B30004B30DD008A1157238A15F808031DA42DA8
:101B40008A11162E8A15EE2EDD01DC014B30840041
:101B50005C0884075D088A11BC208A158000003863
:101B60000319B52DDD0ADC0AA62D3B08DC004B303D
:101B7000DD008A1157238A15F808031DCB2DDC01DF
:101B80005A30DD008A11E5228A157808BB003B082F
:101B9000DC00DD28EE2EDD01DC014B3084005C082A
:101BA00084075D088A11C5208A1580000038031952
:101BB000DC2DDD0ADC0ACD2D3B08DC004B30DD00DE
:101BC0008A1157238A15F808031DF22DDC015A30BB
:101BD000DD008A11E5228A157808BB003B08DC008D
:101BE0009A29EE2EDD01DC014B3084005C0884076D
:101BF0005D088A11D2208A15800000380319032E4F
:101C0000DD0ADC0AF42D3B08DC004B30DD008A11D4
:101C100057238A15F808031D0F2E692BEE2EDD01C0
:101C2000DC014B3084005C0884075D088A11DF20EA
:101C30008A15800000380319202EDD0ADC0A112ED7
:101C40003B08DC004B30DD008A1157238A15F80869
:101C5000031D2E2E0130DC00CF23EE2EDD01DC0132
:101C60004B3084005C0884075D088A11E9208A15DE
:101C70008000003803193F2EDD0ADC0A302E3B08B5
:101C8000DC004B30DD008A1157238A15F808031D4C
:101C90004C2EDC01CF23EE2EDD01DC014B30840025
:101CA0005C0884075D088A11F3208A1580000038DB
:101CB00003195D2EDD0ADC0A4E2E3B08DC004B309A
:101CC000DD008A1157238A15F808031D692E572C49
:101CD000EE2EDD01DC014B3084005C0884075D08DA
:101CE0008A11FF208A158000003803197A2EDD0A38
:101CF000DC0A6B2E3B08DC004B30DD008A115723D9
:101D00008A15F808031D862EB02CEE2EDD01DC01AD
:101D10004B3084005C0884075D088A110C218A1509
:101D2000800000380319972EDD0ADC0A882E3B0854
:101D3000DC004B30DD008A1157238A15F808031D9B
:101D4000A32EDB2CEE2EDD01DC014B3084005C0881
:101D500084075D088A1115218A158000003803194F
:101D6000B42EDD0ADC0AA52E3B08DC004B30DD007A
:101D70008A1157238A15F808031DC62E8A11D3210C
:101D80008A15E6018A11AD228A15EE2EDD01DC01ED
:101D90004B3084005C0884075D088A1121218A1574
:101DA000800000380319D72EDD0ADC0AC82E3B0854
:101DB000DC004B30DD008A1157238A15F808031D1B
:101DC000E92EAA080319E62E0030E72E0130AA00FA
:101DD000EE2E0130E6008A11AD228A158A150A120C
:101DE000532F84011F3083059F308400073080000B
:101DF000A80119308316990026309800903083127C
:101E00009800A901AA01AB01AC01AD01AE01AF017F
:101E1000B001B501B601B701B801B901FF30BA0090
:101E200007113A113A088316870083128710BA10F7
:101E30003A0883168700831205128316051283124F
:101E400085128316851283120530F700F71D302F97
:101E500007308101813084000008C0390F388000CC
:101E60006400813084000008C039770480008A1142
:101E7000CD218A158A11D3218A15831686168312DD
:101E8000861A442F0130B0008A11E2298A157A0897
:101E9000AE007908AD007808AC007708AB008B166F
:0A1EA000C0308B04E92C522F6300C0
:02400E00F13788
:00000001FF
